:100000000C9416090C9431090C9431090C943109A3
:100010000C9431090C9431090C942A0C0C9431097C
:100020000C947A0C0C9431090C9431090C9431091C
:100030000C9431090C9431090C9431090C94310958
:100040000C9431090C9431090C9431090C94310948
:100050000C94310910484947482053434F524510EA
:1000600000464C41534800454550524F4D004E6F9D
:100070007620203120323030380030303A31353A75
:100080003137004F4B004641494C004F4B000103B4
:10009000040404FA0102030303C8010102020296E8
:1000A00001010202026401010202023201010202A4
:1000B00002030264026E02780282028C029602A09F
:1000C00002AA02B402BE02C802D202DC02E602F0B8
:1000D00002FA00028C0A00028C0200028C02000F5D
:1000E000460002DC026E040002DC056E0001A00185
:1000F0008C01780164015001640178018C01A00039
:1001000001C80196016401FA01C8000164015001AF
:100110003C013201640150013C0132016401500193
:100120003C0132000348D225703226306E27181465
:100130002860642901022A11022B01152C111501D6
:10014000050307020604081B1111111111111111E9
:100150001611111111111111111A10232323232328
:100160002323211023232323232323211010211BA6
:100170001A211B111A2110211B111A211B1A2110DF
:1001800010211D1C211D111C2112211D111C211DBE
:100190001C2110102323232323232323232323235E
:1001A00023232323211010211413211521141116A8
:1001B000111321152114132110102323232110239F
:1001C0002321102323211023232321101D11111A71
:1001D00021171113211221141118211B11111C2098
:1001E000202010211023232323232321102110203A
:1001F00020201111111C2112211B1320141A21126D
:10020000211D111111202020232323211020202023
:1002100010232323232020201111111A2115211D21
:100220001111111C2115211B111111202020102149
:1002300010232323232323211021102020201B11EE
:10024000111C21122114111611132112211D11113B
:100250001A1023232323232323211023232323239F
:10026000232321101021141A2114111321122114F7
:100270001113211B132110102321102323232323C7
:1002800023232323232110232110171321122115A7
:1002900021141116111321152112211418102323D2
:1002A0002321102323211023232110232323211072
:1002B00010211411111911132112211411191111E6
:1002C0001321101023232323232323232323232336
:1002D0002323232321101D111111111111111111AB
:1002E00011111111111111111C000000000000006A
:1002F00000000000000000000000000000000000FE
:1003000000000000000000000000000000000000ED
:1003100000006666000666666006660660666666DB
:10032000666660000066666666666666660666669F
:1003300060066666600066660000666600066666C1
:100340006006666660666666666666066666660679
:10035000666606066606660660066606600066064F
:100360000000666600066666600660666066666631
:1003700066000006666666666666666666066666A9
:100380006006666660006666000066060006660631
:100390006006660660660606666666066666660649
:1003A000666666666606666660066666600066661F
:1003B00000006666000660666006666000666000B3
:1003C0000066000000666000006666000006666069
:1003D0000006666660006666000066660006666681
:1003E00060066666606666666660660666666006E5
:1003F000666660006606000060060000600000009F
:10040000000066660006660660000666600000067C
:10041000660000006600000666000066660006666C
:100420006006666660006666000000000006000068
:1004300060060000606660006666600666606606CC
:10044000666666666606666660066666600066667E
:1004500000066666600666666666666666666006CE
:100460006666600666666006666666066666666658
:100470006666606660066000000066666606666620
:1004800066066666660666006606660066066600BE
:10049000660666666606666666066600660066004E
:1004A0006600006666600666006006660060666656
:1004B00066606666606066600060666660600666CC
:1004C0006660066666000066666000066066006636
:1004D00060666066666000666600006666000066CC
:1004E00066000066666660666066006660600006BC
:1004F0006000660006006660660666606606666006
:1005000066666660666666606666666066606660A9
:10051000666066606600660006666660006666661F
:10052000066666660660066606600666066006661D
:1005300006666666066666660660066606600660AD
:100540000066000660660006666660066666660609
:100550006666666666666666666606666666006601
:100560006666000666660006600100001001000075
:100570001001000010010000100100001001000037
:100580001001000010010000100100001001000027
:100590001000000000111111110000000000000007
:1005A000000000000000000000000000000000004B
:1005B00000111111110000000001000010010000E5
:1005C00010010000100100001001000010010000E7
:1005D00010010000100100001000111100000000C7
:1005E00000000000001111110000000010000000C8
:1005F00010000000100000001000000010000000BB
:100600001011111100000000000000000000111185
:1006100011010000000100000001000000010000C5
:100620000001000000010000000011111100000095
:100630000000000000001111000100001001000086
:100640001001000010010000100100001001000066
:100650001001000010010000100000000011111135
:100660001100000000000000000000000000000079
:10067000000000000000000000000000001000006A
:100680000101000001010000000100000001000064
:100690000001000000010000000100000001000056
:1006A0000001000000010000011000001000000027
:1006B00010000000100000001000000010000000FA
:1006C00010000000100000001000000010100000DA
:1006D00010100000010000000000000000000000F9
:1006E000000000000000000000000000000000000A
:1006F0000011111111000000000000000011111183
:1007000000000000100000001000000010000000B9
:100710001000000010000000100000001010000089
:100720001000000000001111110100000001000084
:1007300000010000000100000001000000010000B5
:100740000001000000010000011000001000000086
:100750001000000010000000100000001000000059
:100760001000000010000000101111110000000026
:100770000001000001010000000100000001000074
:100780000001000000010000000100000001000065
:10079000000011111100000000000000000440449E
:1007A000004440444044444440444444400444449D
:1007B00000044444000044400000444000000400A1
:1007C0000000000000000000000000000000000029
:1007D0000000000000000000000000000000000019
:1007E0000000000000000000000000000000000009
:1007F00000000000000000000000000000000000F9
:1008000000000000000000000000000000000000E8
:1008100000000000000000000000000000000000D8
:1008200000000000000007000000070000000000BA
:1008300000000000000000000000000000000000B8
:1008400000000000000000000000000000000000A8
:10085000070000000700000000000000000000008A
:100860000000000000000000000000000000000088
:10087000000000000000070007000700070000005C
:100880000000000000000000000011110001111123
:10089000100101101011011011110110111111118D
:1008A000111111111111111111111111111010103B
:1008B00011004444000444444004044040440440C3
:1008C000444404404444444444444444444444442C
:1008D0004444444444404040440022220002222236
:1008E0002002022020220220222202202222222272
:1008F00022222222222222222222222222202020DE
:1009000022005555000555555005055050550550C8
:1009100055550550555555555555555555555555DC
:10092000555555555550505055003333000333330A
:100930003003033030330330333303303333333356
:100940003333333333333333333333333330303080
:10095000330000000000020200004224000444446E
:100960004004744440044444400444444004444427
:1009700040004444000000000000000000000006A9
:1009800060000006600000666000006660000666A9
:1009900000000666000066600006660000000000B9
:1009A000000000000002200000022220000022229D
:1009B0000000227720022227200222222002222267
:1009C00020002222000000000000000000002200A1
:1009D000000020244000204744044044444744048D
:1009E0004044440000444400000440000000000073
:1009F0000000000000000000000700070070707099
:100A000070707070707070707007000700000000E8
:100A100000005550000500050000000000700000B7
:100A2000007007000070777000707070700077774A
:100A3000770007070700000777000000700000003C
:100A400000700000007000000070070000707070FF
:100A5000000070700000707070000707070000074A
:100A600007000007070000007007777700777777A7
:100A700070771177717717777177771771777117AB
:100A800071771107717777777107777711001111F7
:100A90001000077000007771000077710000077187
:100AA00000000771000007710000077100077777E9
:100AB00070077777710011111107777700777777D3
:100AC000707711177101100771007777110777712F
:100AD000107711110077777770777777710111119F
:100AE0001107777700777777707711177101107793
:100AF0001100077110000077007700077077777793
:100B00007107777711001111100000770000077747
:100B10001000777710077777107771771077117754
:100B2000107777777077777771011177110000016F
:100B300010777777007777771077111110777770C4
:100B400000777777000111777000007771777777FA
:100B50001177777110011111000777770077777798
:100B600010771111107777770077777770771117F3
:100B70007177100771777777710777771100111107
:100B80001077777770777777710111177100007799
:100B9000710007771100777110007711000077104E
:100BA0000000771000000110000777770077777753
:100BB000707711177177777771077777117711173A
:100BC00070771007717777777107777711001111B8
:100BD000100777770077777770771117717710079D
:100BE00071777777710777777100111771077777CA
:100BF000710777771100111110000000000000004C
:100C0000000003300000033100000011000000006C
:100C1000000003300000033100000011000000005C
:100C200000000000660000666600066666006666F4
:100C300006066600060666006606666666000666C6
:100C4000660000066600000006660000006666009A
:100C50000066666000666666006666666066666672
:100C60006066666660666666666666666666666630
:100C70006600000000000000000000000600000602
:100C80006600066666066666660066666600066656
:100C900066000066660000006666666666666666F2
:100CA00066666666666666666066666660666666F0
:100CB0006066666600666660006666000066000044
:100CC0000003333300333333303311133133100324
:100CD00031011033310003331100033110000011D2
:100CE00000000330000000110000000000000000C0
:100CF00000000000000000000000000000000000F4
:100D000000000000000000000000000000000000E3
:100D100000003330000333330033313330331103F9
:100D20003133100331333333313333333133111330
:100D300031331003310110001133333300333333B7
:100D40003033111331333333313333331133111320
:100D50003033100331333333313333331101111155
:100D60001003333300333333303311133133100076
:100D700011331000003310000033100330333333CD
:100D80003103333311001111103333330033333354
:100D90003033111331331003313310033133100367
:100DA0003133100331333333313333331101111104
:100DB0001033333330333333313311111133333094
:100DC000003333310033111100331000003333335B
:100DD0003033333331011111113333333033333383
:100DE000313311111133100000333300003333104D
:100DF0000033111000331000003310000001100008
:100E000000033333003333333033111331331000E5
:100E100011331000003310333033100331333333C8
:100E20003103333311001111103300033033100339
:100E30003133100331331003313333333133333330
:100E400031331113313310033133100331011000EA
:100E50001100330000003310000033100000331085
:100E60000000331000003310000033100000331076
:100E700000003310000001100000000330000003E8
:100E80003100000331000003310000033100000392
:100E90003133000331333333310333331100111154
:100EA0001033000330331033313313331133333104
:100EB0001033331100333330003313330033103326
:100EC00030331003310110001133000000331000E3
:100ED0000033100000331000003310000033100006
:100EE0000033100000333333303333333101111109
:100EF00011330003303310033133303331333133A6
:100F00003133333331333333313313133133131339
:100F10003133131331011010113300033033100338
:100F2000313330033133330331333333313313331C
:100F300031331033313310033133100331011000DA
:100F40001103333300333333303311133133100390
:100F50003133100331331003313310033133333362
:100F60003103333311001111103333330033333372
:100F70003033111331331003313310033133333332
:100F800031333333113311111033100000011000CD
:100F90000003333300333333303311133133100351
:100FA00031331003313313033133103331333333DF
:100FB0001103333130001111013333330033333334
:100FC00030331113313310033133100331333333E2
:100FD0001133333310331133303310033101100028
:100FE00011033333003333333033111331333300D0
:100FF00011033333000013333033001331333333F1
:1010000031033333110011111033333300333333D1
:1010100010013311100033100000331000003310A2
:1010200000003310000033100000331000000110E6
:101030000033000330331003313310033133100316
:101040003133100331331003313310033133333371
:101050003103333311001111103300033033100307
:1010600031333033313331333103313311033133E1
:1010700010033333100033311000333100000111FD
:1010800000330003303310033133130331331313B0
:10109000313333333133333331333133310331335C
:1010A00011033133100011011033000330331003EA
:1010B00031333033310333331100333110033333E1
:1010C0000033313330331103313310033101100059
:1010D00011330003303310033133303331033333F2
:1010E000110033311000333100003331000033314F
:1010F0000000333100000111003333333033333318
:1011000031331133310113331100333110033311F3
:101110000033311330333333313333333101111171
:101120001175021802050075022E000500EA045C24
:10113000000100EA045C00300175022E0005007514
:10114000021802050075022E000400EA042E0001B8
:1011500000EA045C00300175025C00010075022E9B
:1011600000050000000000000050414C00090A0B7F
:101170000C0D0E0F004352454449545320004C457A
:1011800056454C2000474554205245414459004C97
:101190004556454C20444F4E4500424F4E55530056
:1011A000494E5345525420434F494E0020201020B1
:1011B00020201020200047414D45204F5645520029
:1011C0001B111111111111111A0010090A0B0C0D2C
:1011D0000E0F10001D111111111111111C00494E9B
:1011E0005345525420434F494E00434F50595249A2
:1011F000474854203230303500414C42455254204B
:1012000053455741524400252020424C494E4B59EA
:1012100000262020434C5944450027202050494EA9
:101220004B5900282020494E4B45590011241FBE20
:10123000CFE5D4E0DEBFCDBF10E0A0E6B0E0ECE843
:10124000F9E302C005900D92A436B107D9F714E076
:10125000A4E6B0E001C01D92AF31B107E1F70C94F4
:1012600040140C9400008091640013C0815080935E
:101270006400A82FBB27FD01E153FC4F9081953FEF
:1012800040F4AA0FBB1FA752BC4FED91FC91908375
:10129000EACF882359F708952F923F924F925F9299
:1012A0006F927F928F929F92AF92BF92CF92DF9276
:1012B000EF92FF920F931F93CF93DF93CDB7DEB7DB
:1012C00023970FB6F894DEBF0FBECDBF6C015B0154
:1012D0003A01E22E302E4090C5035090C603269569
:1012E0002983E8949C012E0D311D88E990E0821736
:1012F00093070CF49C01D7FCFAC02C193D09121677
:1013000013060CF003C1E22E9501230D311D80EF71
:1013100090E0821793070CF49C01B7FCD9C02A19FE
:101320003B09121613060CF0F4C0322E27E0222ED1
:101330002C20C5016AE070E00E948B1C982ED59489
:10134000C794D594C794D594C7944C0C5D1CC50123
:101350006AE070E00E948B1C23E130E0629FA001F4
:10136000639F500D729F500D1124440E551E990C11
:10137000990C00E063010FB606FE07C00894C11C7B
:10138000D11CF301F490F29401E0122D520188E295
:10139000882EF5014081453F08F449C0455F489DCE
:1013A000900111248091CB039091CC03280F391F19
:1013B0003B832A832A813B81290D311D812F86950C
:1013C000280F311D3B832A83F9019081183028F5BD
:1013D000212F3327A90100FD05C0F6010894C11C87
:1013E000D11CF490F2948F2D8F7021F040FF54C0E7
:1013F000907F982B0F5F0E1508F051C020FF06C09C
:10140000EA81FB819193FB83EA8390811F5F4F5FA9
:101410005F4F2F5F3F4F1830F0F210E00894A11C8F
:10142000B11CE894F5014081453F08F0B7CF8091A9
:1014300064008A3008F049C0E82FFF27DF01A1537C
:10144000BC4F4C93EE0FFF1FE752FC4FB182A082BE
:10145000889DF00111248091CB039091CC03E80F7B
:10146000F91FFB83EA832091C3033091C403489D95
:10147000C0011124820F931F48E250E0BC01CF014C
:101480000E942C1C80916400982F9B508F5F80934A
:101490006400F50190838ECF9F708295AACFEA8178
:1014A000FB819083F9816F0E711C24E0920E37E26C
:1014B000391528F4992443E150E0440E551E3A941E
:1014C00009F057CF80E090E026C081E090E023C093
:1014D0004981842F9927A89EF001A99EF00DB89EFE
:1014E000F00D11246E1A7F0AAA24BB241ACF882774
:1014F00099278C199D099595879518F42F5F3F4F73
:101500006894680E791ECC24DD24F9CE82E090E048
:1015100002C083E090E023960FB6F894DEBF0FBEC2
:10152000CDBFDF91CF911F910F91FF90EF90DF9092
:10153000CF90BF90AF909F908F907F906F905F9073
:101540004F903F902F900895282F3091650083E0B1
:10155000389FD0011124A351BC4F213F60F5E22FE9
:10156000E60FF12DF11DE13FF10564F42C93FD012F
:1015700061834283832F8F5F833070F01092650008
:10158000CD01089560EF621B2C93FD0161834283BE
:10159000832F8F5F833090F7809365009927FC013C
:1015A000EE0FFF1FE80FF91FE351FC4F8FEF818310
:1015B0001282CD01089580E090E0089510926500B8
:1015C00080EF8093EE0388EF8093EF038DEE93E03E
:1015D0009093C8038093C7038091ED036AE00E9453
:1015E0006B1C93E1899FC00111242091C5033091A8
:1015F000C603820F931F9093CA038093C903089573
:10160000FC01962F82818F70907F892B82830895B1
:10161000FC01962F8281887F9770892B828320819D
:101620003AE0822F632F0E946B1C291B842F0E949B
:101630006B1C290F20830895A091C503B091C603A8
:101640004091CD037091CE035091C3039091C40398
:101650002DEC829F212D26952695269533E1239FFB
:10166000A00DB11D3AE0239F8019880F880F112427
:10167000580F911D480F711D28E23D91329FF001D6
:101680008D91829F855F689418F0040E171E03C029
:10169000050E191EE89488E068E021E1355FA8F5A1
:1016A000E50FF91F8695359138F000C003C00000A2
:1016B0003BBB35918A953BBB3295C9F7BEF1000023
:1016C0003BBBF00105900BBA88E23D9102940BBA46
:1016D000082E85918BBB8295E894309D8BBB8591BC
:1016E000355F8BBB359182958BBBD0F5050E191EEE
:1016F000F0013BBB2A95329519F762503BBB20F0B5
:1017000035913BBB3295C9F73BC0E40FF71F869577
:10171000319140F0000003C000003BBB319100005C
:101720008A953BBB3295C1F75EF600003BBBE8945F
:10173000F00181918BBB000038E2032E82958BBBB8
:1017400081913D918BBB8295309D355F8BBB8191A3
:1017500031918BBB8295F00138F200008BBB00C049
:10176000040E171E3BBB2A95329501F7F0013BBBD7
:10177000625028F031913BBB00003295C1F7000068
:101780002BBB112408958FEF83BD8DE185BD13BC64
:101790008F9A08959093F7038093F60381E08093E6
:1017A000660008951092660013BC0895809166004B
:1017B0008823B1F0282F215089F48091F60390916D
:1017C000F703FC0101963491332359F4209366000A
:1017D0009093F7038093F60323BD0895209366004A
:1017E00008953093660001969093F7038093F60373
:1017F0000197FC01849183BD0895909160009F70D2
:10180000807F982B9093600008959093F9038093C4
:10181000F8039093FE038093FD031092000410924E
:10182000FF0382E38FBD89E18EBD84E089BF87ED30
:1018300090E09BBD8ABD8C9A089520E030E0109224
:10184000FC0302C02F5F3F4F8091FC038823D1F33C
:10185000C90108951F920F920FB60F9211242F9372
:101860003F934F935F936F937F938F939F93AF9328
:10187000BF93EF93FF938091FB0383FD1FC0809183
:10188000FF03909100040197909300048093FF035D
:10189000892B51F08091FA038F5F8093FA03803F88
:1018A000C1F48093FB0315C081E08093FC030E9488
:1018B000D60B84E089BF8FEF88BF0BC000904C002F
:1018C00000FE00C06091FB038091FA030E941C0B94
:1018D000D6CFFF91EF91BF91AF919F918F917F9163
:1018E0006F915F914F913F912F910F900FBE0F908D
:1018F0001F9018951F920F920FB60F9211242F93DD
:101900008F939F93EF93FF9380916800909169006C
:1019100097BD86BD8091FF03909100040097D9F494
:10192000E091FD03F091FE0304C0E091F803F09113
:10193000F903859195910097C1F390936900809385
:1019400068008591959199BD88BD85919591F09399
:10195000FE03E093FD030197909300048093FF033F
:101960008950914079F4809167008093FA038091C7
:1019700060008093FB03807F88608ABB80E189BF21
:101980008FEF88BFFF91EF919F918F912F910F90D3
:101990000FBE0F901F9018950F931F93CF93DF9357
:1019A000CDB7DEB725970FB6F894DEBF0FBECDBF1B
:1019B00080E5898381E48A8383E48B8350E09E0100
:1019C0002F5F3F4F0FE010E068EE73E045E0C80185
:1019D000851B9109869FF001879FF00D969FF00D62
:1019E0001124FD83EC83E199FECF549FD001112493
:1019F000F901142E0E94AD1C5F5F5F3040F3259605
:101A00000FB6F894DEBF0FBECDBFDF91CF911F910F
:101A10000F910895CF93E091CB03F091CC0380E533
:101A200011928A95E9F750E075EF66EFC1E1A52FB5
:101A3000BB27CD0120E030E04BE0E091C503F09101
:101A4000C603E80FF91F7083E091C503F091C60348
:101A5000E20FF31FEA0FFB1F638B41502A5D3F4FDC
:101A6000869647FFEACFE091C503F091C603EA0FDF
:101A7000FB1FC0838091C5039091C603A80FB91FB7
:101A8000AB54BE4FCC935F5F533188F2A091C50336
:101A9000B091C603A05BBF4F24E530E001C08D9339
:101AA000F9012F5F3F4F84918823C9F721E180E03E
:101AB00090E049E0E091C503F091C603E80FF91FFB
:101AC000EC59FF4F2083E091C503F091C603E80F66
:101AD000F91F26AFE091C503F091C603E80FF91F87
:101AE000EC56FE4F20834150019647FFE3CFE09133
:101AF000C503F091C6038BE185AFE091C503F0917A
:101B0000C603ED59FF4F87E18083E091C503F09153
:101B1000C603ED56FE4F8DE18083E091C503F09141
:101B2000C603E85BFF4F8AE18083E091C503F09133
:101B3000C603E259FF4F88E18083E091C503F0912D
:101B4000C603E256FE4F8CE1808340E0A3E1B0E0A3
:101B500070E160E2842F99278A9F90018B9F300D5E
:101B60009A9F300D1124C901E091C503F091C6037D
:101B7000E20FF31FEA58FF4F708320E030E059E096
:101B8000E091C503F091C603E80FF91FE20FF31FC0
:101B9000E958FF4F608351502F5F3F4F57FFF0CF01
:101BA000E091C503F091C603E80FF91FEF57FF4F0F
:101BB00070834F5F4F3070F2CF9108952091CB0327
:101BC0003091CC03205B3F4F8CB39927DC01A2708E
:101BD000B07081FDF9CF8BE4F901182E0E949E1C94
:101BE000C90108953F924F925F926F927F928F92B8
:101BF0009F92AF92BF92CF92DF92EF92FF920F939C
:101C00001F93CF93DF93EC010E94DE0D5C010E94D5
:101C10000A0D26E430E0A20EB31EF5018381948103
:101C20002AEB3FEFA20EB31EC817D90768F1FEE0FA
:101C30003F2EEEE04E2E512CC201880F991F880FC7
:101C4000991F840D951D8A0D9B1DDC011596FC01C5
:101C500085E001900D928150E1F73A9437FC12C073
:101C6000432C552447FC5094F201EE0FFF1FEE0F5A
:101C7000FF1FE40DF51DEA0DFB1D83819481C8173C
:101C8000D907D0F6339402C05FE0352E432C55249B
:101C900047FC5094F201EE0FFF1FEE0FFF1FE40D03
:101CA000F51DEA0DFB1DD483C38381E4808381830A
:101CB0008283CC243FE0331609F4DDC06C2C7724FA
:101CC0004201880C991C880C991C840C951C8A0C68
:101CD0009B1CC39484E1C81609F48EC083B380951D
:101CE0008F73871589F0782E99278830910509F42C
:101CF000A9C0893091050CF081C08130910509F4AB
:101D000083C0049709F4B2C0EE24FF24E5018701E3
:101D10009EE0D92EE091C503F091C603E00FF11FBC
:101D2000E958FF4F88818083E091C503F091C60395
:101D3000E00FF11FE858FF4F89818083E091C503D0
:101D4000F091C603E00FF11FE758FF4F8A818083AF
:101D50008091C5039091C6038E0D9F1D84589F4F9F
:101D6000BC018B819C810E940210DA940D5E1F4F92
:101D7000259623E130E0E20EF31ED7FECBCF3EE006
:101D800033150CF47BC0A62DBB2783E190E0489E61
:101D9000F001499EF00D589EF00D11248091C5036D
:101DA0009091C603E80FF91FEA0FFB1FE958FF4F98
:101DB0000C2D112703FF65C0A80DB91D8C918083E0
:101DC000000F111F000F111FE091CB03F091CC0306
:101DD000E00FF11F85E081830E941D0C0E941D0C05
:101DE000E091CB03F091CC03E00FF11F1182C3947B
:101DF00084E1C81609F072CFCC2470CF80319105F0
:101E000059F1809709F080CF639492E0961508F01D
:101E10007BCFEFE03E16B9F1E091C503F091C60328
:101E200088EC91E011920197E9F78CB39927DC01D6
:101E3000A270B07081FDF9CF8BE4F501182E0E94DD
:101E4000AD1C21C0F401E60DF11D8081823408F43F
:101E50005BCF8150808358CFF401E60DF11D808166
:101E60008A3508F051CF8F5F80834ECF662009F40A
:101E70004BCF6A9449CF33E0632E21CF0C2D11272D
:101E80009FCF80E29CCFDF91CF911F910F91FF9068
:101E9000EF90DF90CF90BF90AF909F908F907F900A
:101EA0006F905F904F903F900895AF92BF92CF9206
:101EB000DF92EF92FF920F931F93CF930E94DE0D5C
:101EC0006C010E940A0DC0E0FC2EEC2E03E1A02E56
:101ED000B12C21C00C2F1127000F111F000F111F53
:101EE000E091CB03F091CC03E00FF11F85E08183FB
:101EF0000E941D0C0E941D0CE091CB03F091CC03BD
:101F0000E00FF11F118283B3809581FD55C0F8E188
:101F1000FE1508F451C0CF5FC43109F449C08EE00A
:101F20008F15C0F28F2D99278A9D90018B9D300DC2
:101F30009A9D300D1124E091C503F091C603E20F84
:101F4000F31FE958FF4FDC01AA0FBB1FAA0FBB1FED
:101F5000A80FB91FAC0DBD1D8C9180834091C503A6
:101F60005091C603420F531F48585F4FFD018181B6
:101F7000FA0180834091C5035091C603420F531F5D
:101F800047585F4FFD018281FA018083FA9CC001AE
:101F900011242091C5033091C603820F931F8458EA
:101FA0009F4FBC01FD01838194810E94021092CF5A
:101FB000C0E0F394E394B3CFCF911F910F91FF90C2
:101FC000EF90DF90CF90BF90AF9008958091610027
:101FD00090916200AA27BB27BC01CD012DE63EE40B
:101FE00046EC51E40E944C1CDC01CB01875C9F4C09
:101FF00090936200809361006FEF70E00E94771C05
:1020000099270895CF93DF93EC01FB0180E381933F
:10201000819381938193CE016AE070E00E94771CE6
:102020009B01220F331F220F331F220F331F260F56
:10203000371F260F371FC21B2C2F205D208331979F
:10204000EB01672B41F7DF91CF91089584B3807C3A
:1020500084BB85B38F6385BB08950F931F93CF9384
:10206000082FC62F10E01C1758F483B380958023E7
:1020700039F40E941D0C0E941D0C1F5F1C17A8F351
:1020800080E090E01C1711F081E090E0CF911F916B
:102090000F910895E091C503F091C60388EC91E09B
:1020A00011920197E9F7A091C503B091C603549628
:1020B00021E630E001C08D93F9012F5F3F4F8491FD
:1020C0008823C9F7A091C503B091C603979627E668
:1020D00030E001C08D93F9012F5F3F4F8491882339
:1020E000C9F7A091C503B091C603A35BBF4F2EE60D
:1020F00030E001C08D93F9012F5F3F4F8491882319
:10210000C9F7A091C503B091C603A05ABF4F2AE7F3
:1021100030E001C08D93F9012F5F3F4F84918823F8
:10212000C9F7E091C503F091C603E25BFF4F8081E0
:102130008F7D8083E091C503F091C603E15BFF4F83
:1021400080818F7D808340E0A3E1B0E060E070E0BB
:102150009B0123703070842F8695869586959927EC
:102160008A9FF0018B9FF00D9A9FF00D11248091B2
:10217000C5039091C603E80FF91FE20FF31FE55F57
:10218000FE4F405A40834F556F5F7F4F403400F3FE
:10219000A091C503B091C6035B9623E830E001C06F
:1021A0008D93F9012F5F3F4F84918823C9F7E199FF
:1021B000FECFABEFB1E00E94A31CE158FF43D9F082
:1021C000A091C503B091C6039E9626E830E001C0F9
:1021D0008D93F9012F5F3F4F84918823C9F7E199CF
:1021E000FECFABEFB1E081E89FE30C010E94A81C99
:1021F00081E090E00895A091C503B091C6039E963A
:102200002BE830E001C08D93F9012F5F3F4F84919F
:102210008823C9F780E090E00895DF92EF92FF9263
:102220000F931F93CF93DF93CDB7DEB729970FB6E8
:10223000F894DEBF0FBECDBF8C01D62EE091C50352
:10224000F091C6037E010894E11CF11CD701EA520B
:10225000FF4F89E001900D928150E1F7C8010E9483
:10226000391C2091C5033091C603AC01B801C901E6
:102270008A529F4F0E942C1C6FEF8D2D0E942D10B3
:10228000E091C503F091C603EA52FF4FD70189E000
:102290000D9001928150E1F729960FB6F894DEBFB8
:1022A0000FBECDBFDF91CF911F910F91FF90EF90A7
:1022B000DF9008954F925F926F927F928F929F92DC
:1022C000AF92BF92CF92DF92EF92FF920F931F9344
:1022D000CF93DF935C01E1E0CE2E73E1672E712C8A
:1022E0005C2CEC01259661E0E62EF12C52E0452EA7
:1022F0002981822F6AE00E946B1C992309F0A6C2F3
:102300003881832F992787709070892B09F09EC29E
:102310008A818D3209F419C1F501108101813834A7
:1023200009F46EC1F3E0CF1609F47CC08A818D32C6
:1023300009F478C00E94E60F23E0622F0E946B1C14
:10234000992309F46CC18881181708F02BC25C82AC
:102350008981081708F09CC183E08C838A818432CC
:1023600009F449C14C81423009F4F2C0433009F408
:102370004CC1413009F496C1442309F067C2D880AA
:102380002D2D3327285F3F4F359527953595279578
:10239000359527955981852F6AE00E946B1C9927F6
:1023A00063E1862E912C889DF001899DF00D989D0A
:1023B000F00D1124E20FF31F0091C5031091C60325
:1023C000E00FF11FE0818E2F9927807F907080971A
:1023D00009F42FC1E53F08F02CC1D694D694D694C9
:1023E000852F99270A966AE070E00E948B1C689DF1
:1023F000F001699DF00D789DF00D1124ED0DF11D9A
:10240000E00FF11FE0818E2F9927807F90708097D9
:1024100019F0E53F08F4F6C18B81833009F4F2C16D
:102420004B8214C2F701EF5FFB4F808182958F7062
:1024300009F094CF2881121708F4FDC028812117D4
:1024400058F58B81813041F13327285F3F4F359517
:102450002795359527953595279589816AE00E94BE
:102460006B1C9927869DF001879DF00D969DF00DC0
:102470001124E20FF31F8091C5039091C603E80F6A
:10248000F91FE0818E2F9927807F9070809709F443
:1024900007C1E53F08F004C19981091740F58B8118
:1024A000823029F12881269526952695892F99270E
:1024B0000A976AE070E00E948B1C669DF001679DA0
:1024C000F00D769DF00D1124E20FF11D8091C503F2
:1024D0009091C603E80FF91FE0818E2F9927807F26
:1024E0009070809709F438CFE53F08F035CF998197
:1024F000901708F082C18B81833009F47EC1288156
:10250000269526952695892F99270A966AE070E0E8
:102510000E948B1C669DF001679DF00D769DF00D6D
:102520001124E20FF11D8091C5039091C603E80FBD
:10253000F91FE0818E2F9927807F9070809719F086
:10254000E53F08F45AC14C8209CF18E40EE6EACE02
:102550003881232F269526952695D9808D2D99276C
:102560000A966AE070E00E948B1CA3E1B0E06A9FCB
:10257000F0016B9FF00D7A9FF00D1124E20FF11D19
:102580000091C5031091C603E00FF11FE0818E2F6B
:102590009927807F9070809709F44BC0E53F08F041
:1025A00048C0232F3327285F3F4F35952795359512
:1025B0002795359527958D2D6AE00E946B1C9927EC
:1025C0008A9FF0018B9FF00D9A9FF00D1124E20F6E
:1025D000F31FE00FF11FE0818E2F9927807F90700D
:1025E000809719F0E53F08F4AFC08B81813009F482
:1025F000ABC01B822BC14C814F5F43704C83B3CE69
:102600002E3609F08FCE02E38DCE3881232F26950A
:1026100026952695D9808D2D99270A97A2CF898155
:10262000081708F0BAC02C8388811817B0F55C82AF
:1026300095CE4B830BC18B81882309F4FFCE3327C2
:102640002850304035952795359527953595279510
:1026500089816AE00E946B1C9927869DF001879D05
:10266000F00D969DF00D1124E20FF31F8091C5032C
:102670009091C603E80FF91FE0818E2F9927807F84
:1026800090708097A1F2E53F08F4D8CE5C8266CEC8
:10269000801708F063CE4C8261CE811708F05ECEC1
:1026A0001C825CCED8802D2D3327285030403595A4
:1026B000279535952795359527955981852F6AE07A
:1026C0000E946B1C9927E3E18E2E912C889DF001CE
:1026D000899DF00D989DF00D1124E20FF31F0091DC
:1026E000C5031091C603E00FF11FE0818E2F9927DB
:1026F000807F9070809709F49CCFE53F08F099CFD8
:10270000D694D694D694852F99270A976AE070E0DC
:102710000E948B1C689DF001699DF00D789DF00D65
:102720001124ED0DF11DE00FF11FE0818E2F99278F
:10273000807F9070809711F0E53FC8F18B818230E7
:10274000B1F183E08B8382C08881282F3327285002
:10275000304035952795359527953595279589816D
:102760006AE00E946B1C9927869DF001879DF00D01
:10277000969DF00D1124E20FF31FE00FF11FE08191
:102780008E2F9927807F9070809711F0E53F90F110
:102790008B81882379F15B8259C0801708F044CF80
:1027A0004C8242CF811708F0D3CD1C82D1CD288135
:1027B000269526952695898199270A966AE070E0E4
:1027C0000E948B1C669DF001679DF00D769DF00DBB
:1027D0001124E20FF11DE00FF11FE0818E2F9927E8
:1027E000807F9070809711F0E53F20F08B818330DF
:1027F00009F016CE84E08B8329C00E94E60F837017
:102800008C83ACCD2881269526952695898199279C
:102810000A976AE070E00E948B1C669DF001679D3C
:10282000F00D769DF00D1124E20FF11DE00FF11F68
:10283000E0818E2F9927807F9070809711F0E53F7F
:10284000C8F28B818230B1F283E07CCFC3940894CC
:10285000E11CF11C259684E08C1508F049CDDF9130
:10286000CF911F910F91FF90EF90DF90CF90BF908D
:10287000AF909F908F907F906F905F904F90089552
:10288000C7E5D4E0DEBFCDBF81E291E10E94050C37
:1028900089EE92E09093C4038093C303BAE6EB2ED3
:1028A000B0E0FB2EF092C603E092C50382E392E013
:1028B0009093CC038093CB03885496429093CE039D
:1028C0008093CD0378940E9426100E944A10813094
:1028D00011F40E94CC0CA091C503B091C603AA5775
:1028E000BF4F89E691E1FC0101962491222311F06A
:1028F0002D93F9CF0E94C30B83B3809599278F73D3
:102900009070892BC9F40E941D0CF6CF0E941D0CFB
:102910000E941D0C0E941D0CF394FFEFFF1609F09E
:10292000D7C583B38095992783709070892BC9F799
:1029300089819A810E94F20D0E94961AA1E08A2E46
:102940001A821982F3E09F2ED82C43E050E05C837A
:102950004B83E091C503F091C60388EC91E011929E
:102960000197E9F788EB8093C2038091C5039091AA
:10297000C60342EA51E067E471E043960E942C1CD2
:10298000A091C503B091C603A654BE4F8DE691E158
:1029900001C02D93FC01019624912223D1F763E11C
:1029A00070E04FE050E033E0FA01EB5DFE4F249120
:1029B000FA01EA5DFE4F84919927869FD001879F97
:1029C000B00D969FB00D1124A20FB11D8091C503CB
:1029D0009091C603A80FB91FFA01EC5DFE4F8491D8
:1029E0008C9331504D5F5F4F37FFDECFA091C50311
:1029F000B091C603119685E791E101C02D93FC01CA
:102A0000019624912223D1F7E091C503F091C603EA
:102A100050E3850E818660ED860EA091C503B091CE
:102A2000C6031B968EE791E101C02D93FC01019630
:102A300024912223D1F7E091C503F091C60370E3FE
:102A4000D70ED18A80EDD80E8091C5039091C60330
:102A50008E539E4FBC0189819A810E9402104B8146
:102A60005C814150504080E090E0E3E0FE2EE09138
:102A7000C503F091C603E80FF91FEA54FE4F84170F
:102A800095070CF0ADC32EE12083FA940196F7FE72
:102A9000EECF992009F42DC44D2C4A9473E0572EA3
:102AA00061E085E891E10E940D110E943309509286
:102AB000090420E030E0A6E0B4E043E050E064E048
:102AC000C62EF901EC5DFE4F8491FD018283F90170
:102AD000EB5DFE4F84918C93F901EA5DFE4F84918A
:102AE000FD018183CA941596240F351FC7FEE9CFD7
:102AF00035E0C32E942DC41408F49C2D86E0989FD5
:102B000090011124F901E257FF4F94919F70809139
:102B10000104807F892B80930104F901E157FF4F65
:102B200094919F7080910204807F892B809302048E
:102B3000F901E057FF4F94919F7080910304807FCB
:102B4000892B80930304F901EF56FF4F94919F70F6
:102B500080910404807F892B80930404F901EE5650
:102B6000FF4F94919F7080910504807F892B809303
:102B70000504F901ED56FF4F8491282F332740912A
:102B80000604469546954695809107046AE00E94A2
:102B90006B1C992763E170E0869FF001879FF00D21
:102BA000969FF00D1124E40FF11D8091C5039091C3
:102BB000C603E80FF91F80E28083662477241B0197
:102BC000220F331FA901409550955E834D836BE31F
:102BD00070E0621B730B78876F8383B380959927AE
:102BE0008C7390708830910509F48BC289309105FF
:102BF0000CF07DC2049709F436C386E094E00E948D
:102C00005A1126E0A22E24E0B22E40910704842F10
:102C10006AE00E946B1C992309F00AC20091060425
:102C2000202F3327C90187709070892B09F000C2CB
:102C300010910A04112309F011C3285F3F4F359505
:102C400027953595279535952795842F0E946B1CE0
:102C50009927829DF001839DF00D929DF00D112426
:102C6000E20FF31FE090C503F090C603EE0DFF1DC9
:102C7000E0818E2F9927807F90708097C1F1E53F8A
:102C8000B0F5113009F406C3123009F48CC31330C7
:102C900009F4ABC311E0A12E14E0B12E06E014E05C
:102CA00044E017C0F5018081282F22952F70922FC4
:102CB0009F5F9295907F8F70892B80838F702817EC
:102CC000C9F041500B5F1F4F0894A11CB11C47FD78
:102CD00052C0F80181818E3629F78081813009F454
:102CE000D0C18F38F9F682E0F8018083DBCF1093F2
:102CF0000904D0CFF8018381882309F05BC180816A
:102D0000282F3327C90187709070892B21F5285F00
:102D10003F4F359527953595279535952795818191
:102D20006AE00E946B1C992763E170E0869FF001C6
:102D3000879FF00D969FF00D1124E20FF31FEE0D0B
:102D4000FF1DE0818E2F9927807F9070809719F06A
:102D5000E53F08F42FC1F80180818F5F8083F50182
:102D600080818F70808341500B5F1F4F0894A11C9E
:102D7000B11C47FFAECF42EC51E0E40EF51EB701A7
:102D800089819A810E9402100E941D0C0E943309C1
:102D900000910604802F869586958695282F3327E7
:102DA00040910704842F6AE00E946B1C9927A3E1DD
:102DB000B0E08A9FF0018B9FF00D9A9FF00D1124D7
:102DC000E20FF31FE090C503F090C603EE0DFF1D68
:102DD000808199278332910509F4A6C18432910537
:102DE0000CF052C181973CF0802F9927877090702A
:102DF000892B09F4C6C26114710409F445C0089412
:102E00006108710833E1B30168707070A1E0B0E24D
:102E10004FE050E0E3E0CE2EFA01EB5DFE4F9491DF
:102E2000FA01EA5DFE4F8491839FF0011124E90FBE
:102E3000F11D8091C5039091C603E80FF91F208111
:102E4000822F99278E7F90708E9709F4F6C0CA94CE
:102E50004D5F5F4FC7FEE0CF51E0C52E64E2EBE06F
:102E6000F4E041E050E09BEF69169FEF790609F42A
:102E7000F1C08281843209F4F8C0C3944F5F5F4F80
:102E8000359684E08C1578F78091C203882309F485
:102E90002CC280910904E82FFF27EE0FFF1F9091AD
:102EA000060480910704890F912D911D96958795B1
:102EB0009695879596958795809590958170907059
:102EC000E80FF91FE15CFE4F84918093080418E23B
:102ED00036E0E32E34E0F32EAA24BB2424E0C22EF5
:102EE000F7018281843239F44F8158856416750662
:102EF00010F463FC09C1F7018281819FA0011124B4
:102F00008091C3039091C403480F591F8181992771
:102F100030810AE028E0BC01832F99270E944C09E8
:102F2000CA9448E250E0A40EB51E65E070E0E60EDB
:102F3000F71EC7FED5CF91E0C92E0BE014E087E263
:102F4000E82E81E0F82EF80181818E3649F18091DA
:102F500006049927F8012081821B910906960D9796
:102F600080F48091070499272181821B910908969A
:102F7000419738F48281843209F434C18D3209F0EA
:102F800082C2C39443E050E0E40EF51E0B5F1F4F76
:102F900054E05C1508F421CEF80181818E36B9F633
:102FA00080818134A0F2803590F6F7018491F80198
:102FB0008283CDCFF8018381813009F4E1C0F8012B
:102FC0008381823009F41BC1F8018381833009F0C9
:102FD000C6CE3181832F6AE00E946B1C992319F5BC
:102FE0002081269526952695832F99270A976AE0B2
:102FF00070E00E948B1CCB0163E170E0869FF001C2
:10300000879FF00D969FF00D1124E20FF11DEE0D3C
:10301000FF1DE0818E2F9927807F9070809719F097
:10302000E53F08F49CCEF80181818250818397CEE0
:10303000E090C503F090C6032DCE6115710511F027
:103040002A27208389EB68168FEF780608F0FFCED9
:10305000B083FDCE8281282F3327CA01849628179A
:10306000390709F00ACF628308CF8D819E818615CA
:10307000970509F002CF94E2C90EC2827CEDC70E1B
:10308000FCCE8EE880830ECE8997049708F0B3CEED
:103090008BE091E00E94CA0B8091C2038150809323
:1030A000C20389819A818C599F4F9A838983209189
:1030B0000604269526952695809107046AE00E94CD
:1030C0006B1C9927829DF001839DF00D929DF00D60
:1030D0001124E20FF11D8091C5039091C603E80F02
:1030E000F91F8EE28083FFEF6F2E7F2E88CE803116
:1030F000910509F4F6C0809709F07FCD10920A047B
:103100007CCD50920A0479CD8091C3039091C40381
:103110008A0D9B1D80569A4F2181622F772730811F
:103120000AE028E0AC01F8CE80910904813009F46E
:103130009EC0842F6AE00E946B1C992309F05BCE2D
:10314000842F0E946B1C99278A9FF0018B9FF00DA2
:103150009A9FF00D1124E20FF31FEE0DFF1D80E288
:10316000808389819A810F969A8389838091C20393
:1031700081508093C20380E091E00E94CA0B3BCE55
:103180008081282F3327C90187709070892B21F502
:1031900028503040359527953595279535952795B5
:1031A00081816AE00E946B1C992763E170E0869F31
:1031B000F001879FF00D969FF00D1124E20FF31F91
:1031C000EE0DFF1DE0818E2F9927807F90708097F4
:1031D00019F0E53F08F4F3CEF80180818150BECDAF
:1031E00020E252CC8DE282838DEE90E00E94CA0BE9
:1031F00089819A8188539F4F9A838983C2CE318176
:10320000832F6AE00E946B1C992319F52081269573
:1032100026952695832F99270A966AE070E00E94EA
:103220008B1CCB0163E170E0869FF001879FF00D5E
:10323000969FF00D1124E20FF11DEE0DFF1DE081B0
:103240008E2F9927807F9070809719F0E53F08F4C2
:10325000BBCEF80181818E5F818381CDE090C50373
:10326000F090C6030ECD81E080930A04C6CC842F73
:103270006AE00E946B1C99278A9FF0018B9FF00DDA
:103280009A9FF00D1124E20FF31FEE0DFF1D81E256
:103290008083B1CD202F3327285030403595279596
:1032A0003595279535952795842F6AE00E946B1CEC
:1032B0009927829DF001839DF00D929DF00D1124C0
:1032C000E20FF31FEE0DFF1DE0818E2F9927807F07
:1032D0009070809719F0E53F08F4D6CCF501138380
:1032E000D9CC82E080930A0488CC83ED90E00E94E0
:1032F000CA0B992009F4B8C0A091C503B091C603C8
:10330000AA52BF4F8FE891E101C02D93FC010196B5
:1033100024912223D1F7A091C503B091C603A250F6
:10332000BF4F8AE991E101C02D93FC0101962491E0
:103330002223D1F7A1E0FA2E0D2D11271AC00E94E9
:103340001D0C8091C5039091C6038F5E9E4F98011E
:10335000220F331F220F331FBC01C901800F911FA1
:103360000E940210F3940D0D111D78EC7F1508F4E6
:103370005DC08F2D877019F782EE90E00E94CA0B16
:10338000DECF069506950695842F6AE00E946B1C99
:103390009927829DF001839DF00D929DF00D1124DF
:1033A000E00FF11DDACE202F269526952695842F45
:1033B00099270A966AE070E00E948B1C629DF001DA
:1033C000639DF00D729DF00D1124E20FF11DEE0DC5
:1033D000FF1DE0818E2F9927807F9070809709F4E0
:1033E0007DCFE53F08F07ACF52CC0695069506953D
:1033F000842F99270A976AE070E00E948B1C629DD7
:10340000F001639DF00D729DF00D1124E00FF11D90
:10341000EE0DFF1DE0818E2F9927807F90708097A1
:1034200009F45CCFE53F08F435CC58CF2D2D332778
:1034300088EE93E0289FF001299FF00D389FF00D52
:103440001124CF0129813A81820F931F9A838983A6
:1034500083B3809580FDFCCF83B3809580FFFCCF44
:10346000D394992009F075CAA091C503B091C60301
:10347000A550BF4F80EA91E1FC01019624912223DF
:1034800031F12D93F9CF82EB90E00E94CA0B9A9410
:10349000692D77277C836B83AB014150504080E0DE
:1034A00090E0B3E0FB2E06C02EE12083FA94019653
:1034B000F7FC28C0E091C503F091C603E80FF91F9F
:1034C000EA54FE4F841795077CF320E2EECFFF24E9
:1034D00083B38095992783709070892B09F021CA56
:1034E000F4FE14C0A091C503B091C603AA52BF4F09
:1034F0008CEA91E1FC0101962491222309F406CA89
:103500002D93F8CF992009F0CBCAF3CEA091C50333
:10351000B091C603AA52BF4F86EB91E1FC01019620
:103520002491222309F4F2C92D93F8CF9F92AF92F0
:10353000BF92CF92DF92EF92FF920F931F93CF93A0
:10354000DF9383B3809599278F739070892BC9F788
:10355000E091C503F091C60388EC91E011920197C8
:10356000E9F7A091C503B091C603589620EC31E16C
:1035700001C08D93F9012F5F3F4F84918823C9F7D4
:10358000A091C503B091C6039B962AEC31E101C01E
:103590008D93F9012F5F3F4F84918823C9F7A09144
:1035A000C503B091C603DE9624ED31E101C08D93D1
:1035B000F9012F5F3F4F84918823C9F7A091C5037C
:1035C000B091C603A359BE4F2EED31E101C08D93DA
:1035D000F9012F5F3F4F84918823C9F7A091C5035C
:1035E000B091C603AB55BE4F2AEE31E101C08D93B9
:1035F000F9012F5F3F4F84918823C9F7A091C5033C
:10360000B091C603A854BE4F29EF31E101C08D939C
:10361000F9012F5F3F4F84918823C9F74CE3C42EF3
:10362000D12C36E4A32EB12C21E0922E83B38095C9
:1036300081FD06C198E2E92EF12CCAE0D0E013E04A
:103640003C2D3C1B832F81508739B8F4992009F019
:103650005BC0E32FFF27AE16BF060CF04EC0809173
:10366000C3039091C403885F984F0AE028E0AC013F
:1036700066E470E0CF010E944C0911502A9688E25E
:1036800090E0E80EF91E17FFDBCFC50101978739DF
:10369000910590F4A3FEBDC0992009F4C3C04091E8
:1036A000C3035091C40348535F4F0AE028E066E427
:1036B00070E0C5010E944C09992009F4A2C0089449
:1036C000C11CD11C0894A11CB11C99E9C916D104D4
:1036D0000CF48EC088ECA82EB12C9BEFC916D10437
:1036E0001CF199240E941D0C0E941D0C0E9433099C
:1036F00083B3809581FF9ECFA3C08091C303909137
:10370000C40380569A4FB1CF8091C3039091C403F4
:103710008E0D9F1D80569A4F0AE028E0AC0166E4AA
:1037200070E0832F9927A7CF88EDC8168FEFD806B2
:10373000CCF6A091C503B091C603A958BF4F27E0AE
:1037400032E101C08D93F9012F5F3F4F84918823AF
:10375000C9F76CE382E00E942D10A091C503B091DF
:10376000C603A657BF4F21E132E101C08D93F90195
:103770002F5F3F4F84918823C9F76CE382E00E945A
:103780002D10A091C503B091C603A356BF4F2AE1E7
:1037900032E101C08D93F9012F5F3F4F849188235F
:1037A000C9F76CE382E00E942D10A091C503B0918F
:1037B000C603A055BF4F23E232E101C08D93F9014A
:1037C0002F5F3F4F84918823C9F768EC82E00E9405
:1037D0002D108091C5039091C60340E550E060E252
:1037E00070E089589F4F0E94421C0E94550FB0CE36
:1037F00086EFC8168FEFD8060CF06FCFAA24BB2433
:103800006CCF0894C108D1088EEF9FEFA80EB91EA7
:103810005CCF992071F04091C3035091C403485D7F
:103820005F4F43CF4091C3035091C403485E5E4F46
:103830003CCF4091C3035091C40348585F4F35CFEC
:10384000DF91CF911F910F91FF90EF90DF90CF907C
:10385000BF90AF909F900895FB01DC0140FF05C031
:1038600002C005900D9205900D9242505040C8F74D
:103870000895FC0105900020E9F7809590958E0F42
:103880009F1F0895DC0140FF03C001C06D936D933D
:1038900042505040D8F70895629FD001739FF001C5
:1038A000829FE00DF11D649FE00DF11D929FF00DD0
:1038B000839FF00D749FF00D659FF00D9927729F07
:1038C000B00DE11DF91F639FB00DE11DF91FBD0192
:1038D000CF0111240895991B79E004C0991F961710
:1038E00008F0961B881F7A95C9F780950895AA1B42
:1038F000BB1B51E107C0AA1FBB1FA617B70710F0DB
:10390000A61BB70B881F991F5A95A9F7809590950C
:10391000BC01CD01089597FB092E07260AD077FD3B
:1039200004D0E5DF06D000201AF4709561957F4F32
:103930000895F6F7909581959F4F089513D00192C1
:103940001A94E1F708950ED0E02D0CD0F02D0895D3
:1039500011D0012C0FD01124089501900BD01A948E
:10396000E1F70895E199FECFBFBBAEBBE09A119697
:103970000DB20895E199FECFBFBBAEBB0DBA119653
:0C3980000FB6F894E29AE19A0FBE089589
:04398C00F80100003E
:00000001FF
